:020000040008F2
:0400000018F09FE570
:04002000880008004C
:100040000120704770B50E4E0E4C82B03500361D43
:1000500005E00100306800F0B9F80C350C36A54217
:1000600009D2706831682A688842F2D1306800216C
:1000700000F0BAF8F1E702B070BC01BC0047C0461E
:100080000C0208001802080000000FE11F00C0E386
:10009000120080E300F021E114D09FE51F00C0E3CF
:1000A0001F0080E300F021E108D09FE508009FE5F4
:1000B00010FF2FE14002010000020100C000080013
:1000C00001C08FE21CFF2FE1044C054D054E064F89
:1000D000AE462047002809D0BE4630474100080000
:1000E000D500080045000800ED000800044C054D4F
:1000F0000020AE462047044C044DAE462047000089
:1001000011010800F7000800BD0108000102080005
:1001100000B500F02FF800F03DF812480068C00666
:1001200006D4114810490968104A0A40026006E0E6
:100130000D480D490968802252020A4302600948AD
:100140000068800606D4084807490968084A0A403A
:100150000260E2E7044804490968802292020A43E7
:100160000260DAE720F4FFFF60F4FFFFFFFFFEFF0D
:10017000FFFFFDFF044801210160044802210160E6
:100180000348F421016070470404FFFF0804FFFFE7
:100190000C04FFFF0248C021890401607047C0467B
:1001A00060F4FFFF7047000010B582B004000094B7
:1001B00069460120FFF7F6FFF9E7000000B581B0BE
:1001C00000F01EF801B001BC0047000010B40300AD
:1001D000002A05D00C78491C1C705B1C521EF9D1FA
:1001E00010BC00B0704700000906090E0300002A89
:1001F00003D019705B1C521EFBD100B07047000089
:10020000014CA64620470000A9010800000000009C
:080210000000010000000100E4
:0400000500080000EF
:00000001FF
